:020000001B28BB
:080008001B2863308C000C2062
:100010008D0B052800000800000000000000000013
:100020000000000000008C0B0C28000008000F08E6
:100030008D000520080083160030810000308B0001
:100040008316003085004330860081178312030138
:1000500085008600FA30900096309100C8309200FA
:10006000FA30920005148510051105308D00052029
:1000700005148514051105308D0005200510851423
:10008000051104308D000520051085140515043078
:100090008D00052005108510051503308D00052005
:1000A00005148510051503308D000520900B3228AE
:1000B00005148510051102308D00052000308500E3
:1000C00003308D00052005108514051102308D00C8
:1000D00005200030850003308D00052005108510B7
:1000E000051502308D0005200030850003308D009D
:1000F0000520910B582805148510051101308D003D
:1001000005200030850003308D0005200510851482
:10011000051101308D0005200030850003308D0071
:10012000052005108510051501308D0005200030D3
:10013000850003308D000520920B7B280514851067
:10014000051101308D0005200030850002308D0042
:10015000052005108514051101308D0005200030A3
:10016000850002308D000520051085100515013031
:100170008D0005200030850002308D0005209E286E
:00000001FF
